:0200000480007A
:100000006F00C004732F2034930F8000630AFF0336
:10001000930F90006306FF03930FB0006302FF038A
:10002000170F0080130F0FFE63040F0067000F000F
:10003000732F203463540F006F004000136E9E53E3
:10004000171F00002320CFFD6FF09FFF732540F1A5
:100050006310050073251030635805000F00F00F82
:10006000130E100073000000130E00009702000032
:10007000938282F973905230735020307350303035
:1000800073504030970200809382C2F7638C020065
:10009000739052109302B01A739022307323203061
:1000A000E39E62F873500030970200009382420191
:1000B00073901234732540F173002030B700008034
:1000C00093D10000B70E0080130E20006398D12951
:1000D000B700008093D11000B70E0040130E30001F
:1000E000639ED127B700008093D17000B70E000146
:1000F000130E40006394D127B700008093D1E00035
:10010000B70E0200130E5000639AD125B70000808D
:100110009380100093D1F001930E1000130E600035
:10012000639ED1239300F0FF93D10000930EF0FF64
:10013000130E70006394D1239300F0FF93D110004D
:10014000B70E0080938EFEFF130E80006398D121BE
:100150009300F0FF93D17000B70E0002938EFEFF64
:10016000130E9000639CD11F9300F0FF93D1E00029
:10017000B70E0400938EFEFF130EA0006390D11FF4
:100180009300F0FF93D1F001930E1000130EB00016
:100190006396D11DB72021219380101293D10000C6
:1001A000B72E2121938E1E12130EC0006398D11B0F
:1001B000B72021219380101293D11000B79E901088
:1001C000938E0E09130ED000639AD119B720212106
:1001D0009380101293D17000B74E4200938E2E245C
:1001E000130EE000639CD117B720212193801012D9
:1001F00093D1E000B78E0000938E4E48130EF000AE
:10020000639ED115B72021219380101293D1F00164
:10021000930E0000130E00016392D115B700008009
:1002200093D07000B70E0001130E10016398D01325
:1002300013020000B700008093D170001383010007
:100240001302120093022000E31652FEB70E0001C3
:10025000130E20016314D31113020000B7000080B5
:1002600093D1E00013000000138301001302120079
:1002700093022000E31452FEB70E0200130E300169
:10028000631ED30D13020000B7000080938010009E
:1002900093D1F0011300000013000000138301004C
:1002A0001302120093022000E31052FE930E10007E
:1002B000130E40016314D30B13020000B70000803B
:1002C00093D170001302120093022000E31852FE33
:1002D000B70E0001130E50016392D1091302000002
:1002E000B70000801300000093D1E0001302120059
:1002F00093022000E31652FEB70E0200130E6001B7
:10030000639ED10513020000B700008093801000A7
:10031000130000001300000093D1F001130212003B
:1003200093022000E31252FE930E1000130E700190
:100330006396D10393504000930E0000130E80018A
:10034000639ED0019300100213D0A000930E000012
:10035000130E90016314D001631CC0010F00F00F55
:1003600063000E00131E1E00136E1E0073000000BB
:100370000F00F00F130E100073000000731000C088
:040380000000000079
:1010000000000000000000000000000000000000E0
:1010100000000000000000000000000000000000D0
:1010200000000000000000000000000000000000C0
:1010300000000000000000000000000000000000B0
:081040000000000000000000A8
:040000058000200057
:00000001FF
